:030000000219FDE5
:03000B000200A848
:03002B000201854A
:03005B0002033964
:030073000203265F
:1000800002030406080C10182030406080040608A3
:100090000C10182030406080A0C00003070F1F051F
:1000A000050D050305030302C2AF306308C2638573
:1000B000798AD2AF32C0D0C0E0206221E525601637
:1000C000E473E525F4C3334009758A00D263F579FA
:1000D00001D4F58AD262D0E0D0D0D2AF32C3E526C7
:1000E000334009758A00D263F57901EEF58AC26260
:1000F000E526F4602F30682520720DD0E0D0D0C204
:1001000095C293C297D2AF32C295C293C297206F65
:100110000C2066097412D5E0FDE57B4290D0E0D05A
:10012000D0D2AF32758A00D263757900C28DD262A7
:10013000211D01C2306805206602D29501C23068D7
:1001400005206602D29701C2306805206602D2936C
:1001500001C2C29430680A2066077412D5E0FDD24D
:100160009501C2C29630680A2066077412D5E0FD78
:10017000D29701C2C29230680A2066077412D5E095
:10018000FDD29301C2C2AFC2AD53E6EFC0D0C0E012
:10019000D2D3D2AFE57A6009E57760057577004183
:1001A000D3757701C2CEE52A6007207449152A214C
:1001B000F67800790020742EE580307E01F430E579
:1001C0000278FF53DACF207E0343DA20307E0343E8
:1001D000DA10C2D8C271E580307E01F430E50279D0
:1001E000FFC3E89970CB306103752A18207403753A
:1001F0002A18885CD27020740DE52B6004152B4101
:100200000643DA01C2D82070024179A85C2061025D
:10021000C270207431C3E894F0400374F0F8E8C46D
:10022000540F28F87984B703024146C313C31387D8
:1002300021200802C313200A06C3C898F8414628A3
:10024000F8500374FFF8C3E895655003E565F88836
:1002500022E52D54066022206B1FE536C333C333DD
:10026000F8E564C313C313F9C3952240028922E859
:100270002522F52250037522FF852224A824C3E5F8
:100280002495614002A8618825E566700241BDC3DE
:10029000E8AA669A5003E8FAE4F9EAC333FBE56892
:1002A000F45B29400D2567F8E56760021567400B90
:1002B00041BD0AC3E5679A5002056778FF8826C2E8
:1002C0006FC3E52694F84002D26FC3E52594404001
:1002D00002D26420CF0AD0E0D0D043E610D2AD32B3
:1002E000C2CF053AE57A6009E57860057578006166
:1002F0001C7578017801E52A6005307402152AC35F
:10030000E55C94014005755F00611C7560007569CE
:1003100000E55F2401F55F5003755FFFD0E0D0D0AA
:1003200043E610D2AD32C2AF53E67F7592FA7593B1
:10033000FFC260759104D2AF32C2AF53E6EFC2ADD7
:10034000C0D0C0E0C0F0D2D3D2AFA8FBA9FCE57A00
:100350006007C3E913F9E813F8C2D830710261AB42
:1003600053DACF207E0343DA10307E0343DA20D203
:1003700071E580307E01F420E502618288278928BA
:10038000A1D853DACF207E0343DA20307E0343DA4C
:1003900010C2D8C271307402A1C47800E580307EEA
:1003A00001F430E502A1C4885CA1AC53DACF207E11
:1003B0000343DA20307E0343DA10C27120610281E8
:1003C0008453DACF207E0343DA10307E0343DA20F1
:1003D000C2D8D27188578958C3E89555F8E995561F
:1003E000F97B007E087A00C3E8948CE994005005FC
:1003F000755B008176882178A2E6A8216055C3E864
:1004000094C8E994005008E4D2E4FB7A0A8151C30D
:10041000E89468E994015008E4D2E3FB7A0F815133
:10042000C3E894D0E994025008E4D2E2FB7A1E813A
:1004300051C3E894A0E994055008E4D2E1FB7A3C6A
:100440008151C3E89498E994085008E4D2E0FB7A1B
:10045000787E00C3E89559FCE9955AFD30E70AEC2F
:10046000F42401FCEDF43400FD755B00C3EC9AED5F
:0D0470009E5003755B018859895A855755C8
:10047D008558567802A1ACC3E89527F8E99528F977
:10048D00307C02A190307B02A190307A02A18920AC
:10049D00750281A7E9FDE8FC81C6E9C313F9E813EC
:1004AD00F8307902A189E9C313F9E813F83078021D
:1004BD00A189E9C313FDE813FC20612CC3EC941C46
:1004CD00ED9402400281DDED701EC3EC94C850180E
:1004DD000529E52970021529C3E529940A5002A1C1
:1004ED00C4755C00D270A1C4E52960021529788815
:1004FD00E6F97400207F087896B90302789EE62409
:10050D00FAFEE43400FFC3EC9EFCED9FFD9208B9AA
:10051D000310A2085007207609D276A12F3076025B
:10052D00C276A2085016B9030DECF42401FCEDF4CB
:10053D003400FD02054978007900A190B90315EC4E
:10054D0033FCED33FDC3EC940AFCED9400FD500437
:10055D007C007D00C3EC94FFED9400400678FF799C
:10056D0000A190EC8572F0A4C5F0A2F733F87900E4
:10057D0040030205AC78FF79000205ACE9C313F91D
:10058D00E813F8307C0EE9600278FFC3E81338F801
:10059D00E43400F9C3E894FFE99400400278FF8841
:1005AD005CD270206102A1C4741FF4552F4BF52F3E
:1005BD00C274EB7002D274752A18307403752A0A4E
:1005CD00306102A1D820740353DAFE207403752B19
:1005DD0006D0F0D0E0D0D0D2AD43E6103279010292
:1005ED0006087903020608790A020608791E020632
:1005FD0008796402060879C80206087817E4D5E080
:10060D00FDD8FAD9F6227A147B7802062F7A107B60
:10061D008C02062F7A0D7BB402062F7A0B7BC80253
:10062D00062F7902E4C296D5E0FDD297D5E0FDC242
:10063D0097D5E0FDD296D5E0FDE920E002D29530C8
:10064D00E002D293E573D5E0FDE920E002C29530DA
:10065D00E002C2937496D5E0FDD9C9EAF8D5E0FD64
:10066D00D8FBDBBEC29622C37C007D0075F0000571
:10067D00F0EA33FAEB33FB50F6EB13FBEA13FAC354
:10068D00E9FFE8FEE89AF8E99BF95004EFF9EEF876
:10069D00B3EC33FCED33FDD5F0DFEDF9ECF822E8EA
:1006AD0089F08A20D2D4F8A9F07B0030F70B7BFFBC
:1006BD00F42401F8E9F43400F9E88520F0A4ADF054
:1006CD00F8E98520F0A4AFF0FEED2EF974003FFAA5
:1006DD007C04C3EA13FAE913F9E813F8DCF48BF0A0
:1006ED0030F70AE8F42401F8E9F43400F9E889F068
:1006FD00C2D4F8A9F02222C3E54113F9E54013F85D
:10070D00C3E54498F8E54599F9500CC3E89480E9A0
:10071D0094FF401602073BC3E8947FE99400500311
:10072D0002073B787F790002073B788079FF884983
:10073D00894A22E5492546F8E54A3547F9854A2093
:10074D00E4300701F43548FA30E709C3EA94F04084
:10075D0015020779C3EA940F500302077978FF79E0
:10076D00FF7A0F020779780079007AF0C3E52495B6
:10077D0061500AC374019524500B020797E54A2076
:10078D00E70E020797E54A30E706884689478A480B
:10079D002278A5E6FAC3E54933F8E54A33F9D1AC39
:1007AD00E930E70BC3E89480E994FF4013E1D1C32E
:1007BD00E8947FE994005002E1D1787F7900E1D18E
:1007CD00788079FFE820E715C3E52398F84009C341
:1007DD00E8940140030207F878010207F8E8F424D1
:1007ED00012523F840030207F878FF884B2278A6ED
:1007FD00E6FAA847A9481206ACE930E70CC3E8941D
:10080D0001E994FF401602082DC3E894FFE9940016
:10081D00500302082D78FF790002082D780179FF29
:10082D00E920E715C3E54B98F84009C3E89401406A
:10083D00030208547801020854E8F42401254BF80A
:10084D00400302085478FF88242278FFC26420698F
:10085D003D206A12D264C3E541940A4009C3E525DF
:0F086D0094405002C26479A1E76023E541601F07
:10087C0074FF8541F0848539F0306A0375F005A466
:10088C00F8C5F0600278FFC3E895645002A864884C
:10089C006322C3E54094C8E5419400E5635003141A
:1008AC0001AF046002F563220208B72275E89022BA
:1008BC007883E6FFE5E820ECF7A8BDA9BE0570C378
:1008CC00E57094084052757000E9FA79A0E760442D
:1008DC00EA7007E571601B0208F2C3E895716010BD
:1008EC00E5715006600C140208FE0460F90208FE63
:1008FC00E571F571C39472401B7561C0C3940440DB
:10090C0013756180C39404400B756140C39404401B
:10091C000375610075BB0822E561F460020561E5B1
:10092C0070B4070375BB1022743279A787F0A4C585
:10093C00F0A2F733F8C3E895614002A861882288D9
:10094C0024882588268864227540007541F022C2CF
:10095C00AF75C820A8CCA9CDAA3A30CF010A75C86A
:10096C0024D2AFC3EA13FAE913F9E813F8AB3BACA2
:10097C003C883B893CC3E89BF8E99C20690A547F7E
:10098C00F9306702417521D2AD3D8A3DF9EA9D549B
:10099C007FFA600478FF79FFAE3EAF3F8B3E8C3F11
:1009AC00A83BA93CC3E89EF8E99FF9C3E54113FBBA
:1009BC00E54013FAE82AF540E93BF541500675404D
:1009CC00FF7541FF411CAA40AB41AC40AD417E04D8
:1009DC007F02C3EB940440021E1FC3EB9408400239
:1009EC001E1FC3ED13FDEC13FCDEF7C3EA9CFAEB00
:1009FC009DFBEF6009C3E913F9E813F8DFF7EA2868
:100A0C00FAEB39FB8A408B4150067BFF8B408B41C4
:100A1C00C3EB94025002D2673069047F03414778DC
:100A2C0092E6FFC3E537948240110FC3E53794A0DB
:100A3C0040010FC3EF940640027F057E02E541C4DE
:100A4C00540FF9E541C454F0F8E540C4540F28F8AC
:100A5C00C3E89EFAE99400FB4009C3EA9402EB94C4
:100A6C000050047A02E4FB41C1AA40AB41EBC4FE46
:100A7C00EAC4540F4EFCC3EA9CFAEB9400FBC3E8A7
:100A8C0013C313F8EA28FAEB3400FB8A408B41C3FA
:100A9C00EB94024002C2677802EBC4FE7B00EAC40E
:100AAC00540F4EFAC3EA98FA4005C3940250027AE6
:100ABC00027892E6FF30600241C1855192855293D3
:100ACC00D26043E680C3E49AF8E49BF9C3E833F8B8
:100ADC00E933F93067026154E8FAE9FBD3E913FD15
:100AEC00E813FC88518952C3EF94036038EF20E07F
:100AFC000DE82CF8E93DF9ECFAEDFB020B1DE828AA
:100B0C00F8E939F9C3E82402F8E93400F97AFE7BF4
:100B1C00FFC3EF9403400E8A538B54884D894E8C3F
:100B2C004F8D506188885389548A4D8B4E8C4F8DD4
:100B3C00503069127553F07554FF754FF07550FFB6
:100B4C007551F07552FF6188E8FAD3E813FC8851AF
:100B5C00C3EF94036020EF20E007E82CF8ECFA6177
:100B6C0074E8282402F87AFEC3EF940340088A53F1
:100B7C00884D8C4F618888538A4D8C4FE568C33300
:100B8C005002646BF5683060026192753402D26079
:100B9C0043E680E52D5406602DA840A941C3E91316
:100BAC00F9E813F8306904E92440F9C2AF53E67F41
:100BBC00759100C3E498F594E499F595759104D278
:100BCC006043E680D2AF22D26575430075200030B9
:100BDC006C03752040020BF2D26575430075204002
:100BEC00306C0375200078017901206720E52D54C5
:100BFC00066002C2657914E541C313700104F8C3A1
:100C0C00941440027814306904781B791BC3E833C0
:100C1C00F8C3E933F9206010E543600C306903D563
:100C2C003404D26D81A9719A0543E59B5440B520DB
:100C3C0002819330690908C3E89940011881212089
:100C4C00650A08C3E899400261F28121C265C2AF0E
:100C5C0053E67F7591003067127594007595FC759D
:0F0C6C009104D26043E680D2AF61F2AE40AF4157
:100C7B00C3EE33FEEF33FF50047EFF7FFFC3E49ED2
:100C8B00F594E49FF595816BC3E5339401500261B4
:100C9B00F230650261F2D80281A78121C26DC2AF29
:100CAB0053E67F7591008553948554957591048512
:100CBB004D92854E93D26043E680D2AFE52D54061C
:100CCB006008206A020533020CE5306D0D206C0ABA
:100CDB002065071581158102158A2278003064057D
:100CEB003065027801E53775F007A4F9E5F028F5D2
:100CFB00F0E9A2F013A2F113A2F213F537C3947823
:100D0B005003753778C3E53795384008D266C295DE
:100D1B00C293C297306002A11F854F92855093D228
:100D2B006043E68022207D16C2AF754202C296D286
:100D3B0094306202D293D2AF759F11020F1FC2AFD4
:100D4B00754202C296D292306202D295D2AF759F93
:100D5B0011020F1F307243207D20C2AF75420390EA
:100D6B000163757B40C293C292306204D297A17D1E
:100D7B00D296D2AF759F13020F1FC2AF754203906D
:100D8B000163757B40C295C294306204D297A19DDA
:100D9B00D296D2AF759F10020F1F207D17C2AF7571
:100DAB00420390013EC293306202D297D2AF759F3D
:100DBB0013020F1FC2AF75420390013EC295306202
:100DCB0002D297D2AF759F10020F1F207D16C2AFB4
:100DDB00754204C294D292306202D297D2AF759F01
:100DEB0010020F1FC2AF754204C292D2943062023E
:100DFB00D297D2AF759F13020F1F307243207D2005
:100E0B00C2AF754205900152757B10C297C29630E6
:100E1B006204D295C123D294D2AF759F11020F1FDA
:100E2B00C2AF754205900174757B04C297C29630B0
:100E3B006204D293C143D292D2AF759F11020F1F9E
:100E4B00207D17C2AF754205900134C29730620204
:100E5B00D295D2AF759F11020F1FC2AF754205908D
:100E6B000148C2973062EBD293D2AF759F11020F3C
:100E7B001F207D16C2AF754206C292D29630620217
:100E8B00D295D2AF759F13020F1FC2AF754206C228
:100E9B0094D296306202D293D2AF759F10020F1F7D
:100EAB00307243207D20C2AF754201900174757B77
:100EBB0004C295C294306204D293C1C9D292D2AF0C
:100ECB00759F10020F1FC2AF754201900152757BC7
:100EDB0010C293C292306204D295C1E9D294D2AFC0
:100EEB00759F13020F1F207D17C2AF754201900132
:100EFB0048C295306202D293D2AF759F10020F1F7A
:100F0B00C2AF754201900134C293306202D295D2C6
:100F1B00AF759F13C26622900132757B00C295C2DA
:100F2B0093C297C294C292C296C26222788076FF15
:100F3B000876FF0876FF0876FF0876030876040824
:100F4B00760A087603087601087601788C76010814
:100F5B0076FF0876FF0876FF0876FF0876FF08769F
:100F6B00030876FF0876FF0876FF0876250876D00B
:100F7B000876FA0876FA0876040876FF08760108F0
:100F8B00760008767A0876FF0876010876010876EF
:100F9B0000087603087600227887E6FFC272BF034B
:100FAB0002D2727888E6C394036008C27DE630E112
:100FBB0002D27DC27E7889E630E102D27EC3EF9405
:100FCB00026008758E01D273020FDB758E00C2733F
:100FDB00227880E6149000809378A5F67881E61449
:100FEB009000809378A6F67886E61490008D93781F
:100FFB00A7F67886E6F539C3940250037539027863
:10100B009CE67538FFB402037538A0B4030375383A
:10101B008278A3E61490009A93F566120F2222228F
:10102B007896E6FA7897E6FB7888E6B40305C3EB87
:10103B00940EFB307F047A007BFFC3EB9AFCC394C6
:10104B008250027C827572000572EC8572F0A4C32B
:10105B00E5F0947D40F222D27F112B1205F97A0034
:0F106B007B007C101205EFE55C2AFA74003BFB5A
:10107A00DCF37C04C3EB13FBEA13FADCF7FEC27F52
:10108A00112B22E5EF20E6037520000520903FFF93
:10109A00E520146006901FFF146000930460037536
:1010AA00EF1253D9BF7581C043FF801205EA75EF6D
:1010BA000243B203E5B3240220E70DF521E5E3205C
:1010CA00E0068521B343E301120F227580FF75A460
:1010DA000075F1B275D4DF75900175A5FC75F2FE45
:1010EA0075D50175A60175E241120F22E4F8F6D80A
:1010FA00FD756801120F371215E4789886737530FA
:10110A0001C2AF1206031206131205F912061A12C9
:10111A0005F91206211205F91216FD120603120626
:10112A00031205FEC2AF78FA79FA308507D9FBD8DF
:10113A00F7021C00120FA3120FDC112A112B789848
:10114A008673120F2275A90075B680757A007588A4
:10115A001075890275C82475910475D84075A8223E
:10116A0075B80275E690759B80759D0075D10E75F0
:10117A00BCC075BB0875BA1175E8801205EAD2AF12
:10118A001208B475360053DACF207E0343DA2030D2
:10119A007E0343DA1043DA01C2D8C271120603D2BF
:1011AA00617B037A0CE55B70077A0CDB0302112E74
:1011BA001205F920700302112EC270E55CC3940275
:1011CA0040E1E52F541F855E5DF55EB55DD5DAD544
:1011DA00C26153DACF207E0343DA20307E0343DA3A
:1011EA0010C2D8C27178A2E67008D274E52F54E012
:1011FA00F52FC2757529001205FE307409C3E52959
:10120A00940A4002D2751205EF780230740278000F
:10121A00C3E55C9840F0C2AF120613120613120619
:10122A0013D2AF120603754C007888E6B403026144
:10123A00111205EF788CE6C394015003021311E5ED
:10124A0030C394015003021311207435C3E55C9432
:10125A00FF5003021311C2AF120628D2AF1205FEC5
:10126A00C3E55C940150EFC2AF1206131205F412E3
:10127A000613D2AF1205FEC3E55C94FF40E90217DC
:10128A00827F05D27F112B1205FEC2AFC27F112BBE
:10129A00AE5CC3E55C947FD2AF40761205EAC2AF7A
:1012AA00120628D2AFDFDC1162C3EE94057897F6F6
:1012BA001206031216261217057F0AD27F112B1265
:1012CA0005FEC2AFC27F112BAE5CC3E55C947FD230
:1012DA00AF50E61205EAC2AF1206131205F412065F
:1012EA0013D2AFDFD61162EE24037896F612060304
:1012FA001216261217341205FE112BC3E55C94FF51
:10130A0050024153021782C3E55C954C4003855C49
:10131A004C1205FE78017988E7B403027805C3E523
:10132A005C9840024133C2AF120628120628120600
:10133A0028D2AF120603753000E4F531F5320531D3
:10134A00E531F4703F0532789AE67819146012781C
:10135A003214600D787D14600878FA1460037532CF
:10136A0000C3E53298401D120F221205EA153275A4
:10137A00310078998673C2AF120628D2AF78988660
:10138A00731205FE1205F4E52A7005307402212E47
:10139A0078012074027806C3E55C9840A17888E653
:1013AA00C3940360031205FEE52A700302112EC2DC
:1013BA00AF120F22E4F522F523F524F525F526F5DB
:1013CA0067D2AF7885E6C333F565E4F544F545F5AC
:1013DA0046F547F548F570F52CF52DF53775700883
:1013EA0075BB101205EA1208B8E5E820ECFBA8BDA7
:1013FA00A9BEE97001F888711208BC75700875BB3E
:10140A0010120FA3C2AF7561FF12093485226185DC
:10141A002262852263D2AF752201752401752501E6
:10142A00752601856069756A0175B69075A9037597
:10143A007A017888E6B40307C27D307602D27DD27B
:10144A0068D269753300120E7C120EAB120954125F
:10145A00095B12095412095B120954120BE41207B0
:0D146A0003120CE6120D3012095B120BD3B9
:10147700306E031207042067031208573067031200
:10148700089E120CE6120D5F12095B120BE4306E18
:1014970003120740120CE6120DD612095B120BD38A
:1014A700306E0312079E120CE6120E0512095B122C
:1014B7000BE4306E031207FB120CE6120E7C1209C6
:1014C7005B1208B8120BD3120CE6120EAB1208BC53
:1014D70012095B30692F856461856462856069756F
:1014E7006A0179187A0CC3E53399400CC269D26A4C
:1014F7008A357561FF02150CC3E55C940140030250
:101507001465021592306A1D206C1AE535147006B1
:10151700C26AD26B8165F535C3E55C94014003026D
:101527001465021592753600788279A4E76002780F
:1015370003C3E55F985054307404E52A604D7888FA
:10154700E6B40317207D05207607A162307602A155
:1015570062206C07D26C85646181A478F0306C05D9
:101567008564617820C3E5419850028165306C1B22
:10157700C26CC27D307602D27DD26A75351285641F
:101587006181650536E55C6002A195753600C2AFDD
:10159700120F227887E6FE7602120FA37887EEF6FF
:1015A700E4F522F523F524F525F526F565752C00D8
:1015B700752D0075A90075B680757A00D2AF120532
:1015C700FE120F2278A4E66006D295D297D2933006
:1015D7007409C3E53694044002212E6143901A0D25
:1015E7007820121668E520B45A0CA3121668E52075
:1015F700B4A503021606120F3712162602162590F7
:101607001A0378807B0A121668A308DBF9901A0F71
:10161700788C7B19121668A308DBF9901A2822C266
:10162700AF1216A7121681901A00740E12166DA328
:10163700740612166DA3741512166D901A0378802E
:101647007B0A12166CA308DBF9901A0F788C7B19AA
:1016570012166CA308DBF91216BA121698901A28FC
:1016670022E493F622E6438F01538FFD75EF02754F
:10167700B7A575B7F1F0538FFE22438F02438F0151
:1016870075EF0275B7A575B7F1901A0DF0538FFC7A
:1016970022901A0D745AD16D901A0E74A5D16D222D
:1016A7007A3079D07820901A40D168E520F709A3DD
:1016B700DAF7227A3079D0901A40E7D16D09A3DAA8
:1016C700F922AB74A875BB01027984BB0202798544
:1016D700BB03027986BB04027992BB05027987BBFB
:1016E700060279A3BB0702799CBB08027988BB096C
:1016F700027989E8F7227C05120603DCFB22C2AFD8
:1017070012061312061A1206211206281205F412DF
:10171700061312061A1206211206281205F41206DB
:101727001312061A120621120628D2AF22C2AF12CE
:10173700062812062112061A1206131205F41206BB
:101747002812062112061A1206131205F412062889
:1017570012062112061A120613D2AF22AE74AF7503
:10176700C2AF1206131206131206131205F4DEF2A5
:101777001206281205F4DFF8D2AF22F105D1FDD108
:10178700FD757401757501757600F1637C05AD5CB7
:10179700120603C3ED955C70F5C3E55C9401400A3E
:1017A700C3E55C94FF40320217BED1C9D126F105CB
:1017B700C2AF75EF12D1FDDCD50576C3E57694038C
:1017C700500280C6D1FD0575E5741490009F93F80B
:1017D70008C3E57598500280AED1FDD1FD0574C3ED
:1017E700E574940A5002809C120F37D126C2AF7558
:0417F700EF12D1FD1F
:0319FD0002108D48
:101A00000E0615FFFFFFFF03040A0301015AA5019B
:101A1000FFFFFFFFFF03FFFFFF25D0FAFA04FF01DE
:091A2000007AFF0101000300FF40
:101A4000234656544C6962656532304150726F23AB
:101A500023424C48454C492346333930232020202B
:101A60002020202020202020202020202020202076
:101C0000C2AFC2D353D9BF7581C043B20343FF8073
:101C1000752438752503B1C975EF0275E24043F1AB
:101C20002053A4DF75D4FFD2857DFA780379E67C52
:101C300010752200752300901DD67B0675249875BB
:101C400025013085028142208508D8FBD9F9DCF7CF
:101C500081B4308508D8FBD9F9DCF781B4B189E4C7
:101C600093A3C39A6004DDC381B4DBDBB17B600264
:101C7000812B7B08E493FAA3B15CDBF87A30B15C8A
:101C8000752200752300B17BEAFCEBFDC3ED94FEE9
:101C9000400EB17B8A278B28ED30E0048A828B834B
:101CA000B17B7AC270D8C3ED94FE601350CEBD00F4
:101CB00025EC60097520007521FF0200008100A855
:101CC00027A9280809D804D90281D3B17FEA89AAB3
:101CD000F281C50D81A0C3ED94035049EDA2E092BD
:101CE000007AC5C3E5829400E583941C50902000DF
:101CF00010438F02438F0175B7A575B7F1F030001F
:101D00001FA827A9280809438F01538FFDD804D99C
:101D100002A12089AAE275B7A575B7F1F0A3A10DBC
:101D2000538FFC817C7AC1BD030CE493A3FAB140CC
:101D3000DCF8B138817C817EAA22AB23B15CEBFA5E
:101D4000EA6222752608C3E52313F523E52213F57D
:101D50002250066323A0632201D526EAB1C9B1C986
:101D600075260AEAF4200102D285300102C285B14B
:101D7000C9C3134002C201D526EB22B17FEAFB2082
:101D80008502A17F308502A184752608AE24AF2587
:101D9000C3EF13FFEE13FEB1CDB1C9C3EA13308513
:101DA000024480FA30E703632201C3E52313F523DD
:101DB000E52213F52250066323A0632201D526D91C
:101DC000E52265236523F52222AE24AF250E0FDE22
:101DD000FEDFFCD20122424C48656C693437316326
:041DE000F390060175
:00000001FF
